:020000040000FA
:02000000F228E4
:08000800CC28A0008101831641
:100010000313C03081050800A0008101831603137B
:10002000C030810501308104831203130B110B1DB5
:100030001728A00B16280800A200E1308605220D23
:100040001E39860408008613262886170613A30087
:100050002308230E1C20332023081C203320E130EA
:1000600086058613080001300C20861686120130A2
:100070000C2008002808A900A7106430A1004B201C
:1000800025200A30A1004B2025200130A100A71413
:100090004B2025200800A00121082902031C552817
:1000A000A00A2108A902A7144D2830302007A71C58
:1000B00020300800B101B2010630B30008008316F9
:1000C0000313981C612883120313990008002A085F
:1000D000AC007C20A71D75282B08AC007C20A71144
:1000E000981C752818121811181627118316031357
:1000F0008C16831203130800C53023202C082520FA
:10010000CD3023202C08A8003A2009305F2072301F
:100110005F2065305F2063305F2065305F2069308D
:100120005F2076305F2065305F2064305F202030B4
:100130005F202C085F2020305F206F305F206E3002
:100140005F2020305F204D305F2069305F206330BA
:100150005F2072305F206F305F2063305F20683037
:100160005F2069305F2070305F2020305F2050308A
:100170005F2049305F2043305F2031305F203630D0
:100180005F2046305F2037305F2037305F200D30F2
:100190005F200A305F2008008B138B1BCC28AD003A
:1001A000030EAE0083010A08AF008A01831304081E
:1001B000B0008C1ADC28E9281A08AA008C1EE32853
:1001C0001A08AB00A7152715831603138C12831288
:1001D0000313300884002F088A002E0E8300AD0E12
:1001E0002D0E09008B01831603130130860583123F
:1001F0000313861206138613E130860504300C20A3
:1002000003301C20332001300C2008301C20332008
:1002100001300C2002301C20332001300C2028300B
:1002200023200C3023200130232008300C2083169B
:1002300003131815193099008312031398178316A6
:1002400003138C169816831203130B171816F83025
:100250008B058C018D018B17A7015230252053305F
:100260002520323025203330252032302520203003
:100270002520433025206F3025206D3025206D301E
:100280002520753025206E302520693025206330EB
:100290002520613025202D302520C03023207430CA
:1002A0002520693025206F3025206E302520203014
:1002B00025206F3025206E3025202030252050301D
:1002C0002520493025204330252031302520363067
:1002D0002520463025203730252037302520303066
:1002E000A40002308A002408303C08225F20A40BBE
:1002F00071291A3005200730132061305F206E30DD
:100300005F2069305F206D305F2061305F20743086
:100310005F2069305F206E305F2067305F202030C3
:100320005F204C305F2043305F2044305F202E3010
:100330005F202E305F202E305F200D305F200A308E
:100340005F201030A40018302320C0300C20A40BF4
:10035000A32901302320523025205330252032306C
:1003600025203330252032302520203025205230E2
:10037000252065302520633025206530252070300C
:10038000252074302520693025206F3025206E30DF
:1003900025203A302520C0302320433025206830E6
:1003A00025206130252072302520C730232056308B
:1003B0002520613025206C302520753025206530C2
:1003C000252072305F2065305F2061305F2064300F
:1003D0005F2079305F202E305F202E305F202E305E
:1003E0005F200D305F200A305F205A2027195A20E5
:1003F00027196720B10BF629B20BF629B30BF629A2
:1004000040305F200D305F200A305F205A20F629EF
:1004100082070D340A344D346934633472346F34D6
:10042000633468346934703420345034493443348C
:1004300031343634463437343734203463346F340F
:100440006E346E346534633474346534643420340B
:1004500061346E34643420347334743461346E34F3
:1004600064342D34623479342E342E342E340D34E9
:020470000A344C
:02400E00F23F7F
:00000001FF
